:1000000000308A000428000084011F30830571300D
:1000100083168F0083121F1383161F109F101F114A
:100020009F110730831299001F1383161F109F1012
:100030001F119F1183121F1083160108C73908383A
:100040008100831290010030A100920000308316DD
:1000500092000515831295019501073099008316CA
:10006000050806308312A000A00B342800001908F0
:100070008C118316990171308F00851083128510C1
:100080001030A000A00B422800008316851002301B
:0800900083128506402863007D
:02400E00C43CB0
:00000001FF
